:020000040000fa
:10000000f01f0020c50e0000c31200004d170000b5
:1000100000000000000000000000000000000000e0
:100020000000000000000000000000003710000089
:10003000000000000000000037100000151600004e
:100040003710000037100000371000003710000094
:100050003710000037100000371000003710000084
:100060003710000037100000371000003710000074
:100070003710000037100000371000003710000064
:100080003710000037100000371000003710000054
:100090003710000037100000371000003710000044
:1000a0003710000037100000371000003710000034
:1000b0003710000037100000371000003710000024
:1000c0003710000037100000371000003710000014
:1000d0003710000037100000371000003710000004
:1000e00037100000371000003710000037100000f4
:1000f00037100000f01f0020c50e0000c3120000e2
:100100004d1700000000000000000000000000008b
:1001100000000000000000000000000000000000df
:100120003710000000000000000000003710000041
:1001300015160000371000003710000037100000bf
:100140003710000037100000371000003710000093
:100150003710000037100000371000003710000083
:100160003710000037100000371000003710000073
:100170003710000037100000371000003710000063
:100180003710000037100000371000003710000053
:100190003710000037100000371000003710000043
:1001a0003710000037100000371000003710000033
:1001b0003710000037100000371000003710000023
:1001c0003710000037100000371000003710000013
:1001d0003710000037100000371000003710000003
:0801e000371000003710000089
:020000040000fa
:1001e800f8b5c046f8bc08bc9e4670475d100000d4
:1001f800f8b5c046f8bc08bc9e46704739100000e8
:020000040000fa
:080208000800000001000000e5
:020000040000fa
:10021000f0b51f0085b005000c0016000092019794
:1002200002900391002f00d0d5e08e424ed93000cd
:1002300000f0bcff58b120232a001b1ada4084408a
:100240001300864085402343009603930295009b4c
:1002500003991a0cb1fbf2f615006b463700754393
:100260001b884d1b5f4302992d040c0c2543310064
:10027000af4208d9009c01392d19ac4203d8af42d6
:1002800001d9b11e2d19ef1bb7fbf2f46243bf1a5f
:100290006a46634312893f043a432600934208d9d1
:1002a000009d013e5219954203d8934201d9a61ee2
:1002b00052190904d31a31430a9a1ab1c340136080
:1002c000002353600800019905b0f0bd1eb9012359
:1002d000b3fbf6f30093009800f068ffc0bb009bef
:1002e000e41a01230193009b1a0cb4fbf2f11600ef
:1002f0006b460d004e431b88a41b5d43029e2404e5
:10030000360c34430f00a54208d9009e013fa419c2
:10031000a64203d8a54201d98f1ea419641bb4fbc1
:10032000f2f67243a41a6a467343128924041443f2
:100330003100a34208d9009a0139a418a24203d877
:10034000a34201d9b11ea4183f04e31a3943b3e70d
:10035000009b20228340009323002f00121ad340d9
:100360008540d740009a0295110cb3fbf1f56a461f
:100370002e0012888440944656430a006a4327435d
:100380009b1a1b043a0c13432a009e4208d9009c76
:10039000013a1b199c4203d89e4201d9aa1e1b197f
:1003a0009e1bb6fbf1f5644669436c43761a36042e
:1003b000bfb237432b00bc4208d90099013b7f18dc
:1003c000b94203d8bc4201d9ab1e7f1812041a43ac
:1003d0003c1b019287e78f4209d90a9b002b00d171
:1003e000a9e0186059600023019319006ae73800fa
:1003f00000f0dcfec8b9a74202d30100ae4208d823
:10040000ae1bb542ad410121e41b6d42631b03935a
:1004100002960a9b0193002b00d153e7029a1a60bf
:10042000039a5a60002301934ce720231b1a009380
:100430003b003700009a8340d7401f432300d3403e
:100440002a0000998440ca40224394463a0cb3fbe8
:10045000f2f41100864085406143019626005b1a44
:1004600061460295bdb26e43090c1b040b4321008b
:100470009e4207d9db1901399f4203d89e4201d918
:10048000a11edb199e1bb6fbf2f462436346b61a4b
:100490006a46654393819289360416432300b54228
:1004a00007d9f619013bb74203d8b54201d9a31ebb
:1004b000f619090419436b469c88019b721b9446ec
:1004c0001a0c23008eb20d0c6c43734355437243d8
:1004d0001e0c1219b218944202d9802464022d19fc
:1004e000140c9bb212046519d218ac4503d30bd17e
:1004f000029b934208d2019bed1bd61ab242924155
:100500005242ad1a320001390a9b0193002b00d1ef
:10051000d8e6029b009c9a1a63465d1b029b93429d
:10052000bf417f42ed1b2b00c240a340c5401a4390
:0a0530000a9b24c376e70a9b56e7f6
:020000040000fa
:02053a00704708
:020000040000fa
:10053c0070b505000e0000682b005a1e9341040094
:10054c00621e94411c40f4b301b93a4e03019e4221
:10055c003bd3010b00053200002300f087fd802304
:10056c005b02181a0021002862d0334a1368022655
:10057c00b3431360d369002bfcd180b22e4b98810e
:10058c006b68022b42d02c4a136849032b48184045
:10059c0080235b040343194311605168ab68e8681e
:1005ac000343274801400b4369680b435360224abd
:1005bc00d369002bfcd1204a136802210b43136032
:1005cc00d369002bfcd1200070bdc3009e420ad31e
:1005dc00410bc0043200002300f048fd80235b0275
:1005ec00181a0221bfe743001b189e421ed3c022db
:1005fc0092020023002100f0f7fc3200002300f0ef
:10060c0035fd80235b02181a0421ace70a4a1368f3
:10061c0049030a480340194311605168ab68e86804
:10062c000343072081430b435360c0e70024cae710
:10063c000024c8e70048e801000c0042ff1ffff04f
:04064c00f8dfffffd5
:020000040000fa
:10065000f7b58a8905000c0013075ed44b68002ba0
:1006600004dc0b6c002b01dc0020febde76a002fd0
:10067000fad000232e682b6041f200031a4092b397
:10068000606da3895b0705d56368c01a636b0bb106
:10069000236cc01a0200216a00232800e76ab847c9
:1006a000a189431c06d12b681d2b30d82b4ada4078
:1006b000d3072cd50023636023692360cb0404d5c2
:1006c000431c01d12b6803b96065616b2e60002962
:1006d000cad023004433994202d0280000f094fa93
:1006e00000206063c1e70123216a2800b847431c4a
:1006f000c7d12b68002bc4d01d2b01d0162b01d1e4
:100700002e60b1e74023a2891343a381ade74023c4
:100710000b430120a3814042a7e70f69002fa3d01c
:100720000b680f60db1b01930023920700d14b691c
:10073000a360019b002b00dc96e7019b3a00216a35
:100740002800a66ab047002803dc4023a28913438f
:10075000dfe7019b3f181b1a0193eae701004020e5
:020000040000fa
:10076000344b70b51d6806000c0025b1ab6913b998
:10077000280000f04bfb304b9c420fd16c680c23df
:10078000e25e93b219072cd4d90611d40923336041
:10079000402301201343a381404270bd274b9c425c
:1007a00001d1ac68ebe7264b9c42e8d1ec68e6e768
:1007b0005b0712d5616b41b123004433994202d0eb
:1007c000300000f021fa002363632422a3899343bd
:1007d000a38100236360236923600823a289134354
:1007e000a38123695bb940f2802140f20022a389f2
:1007f0000b40934203d02100300000f0cbfa0123dc
:10080000a28913408bb10023a36063695b42a3619b
:1008100023690020002bc0d10c23e25e1306bcd557
:1008200040231343a3810138b7e7920700d46369db
:10083000a360ede78c000020741500009415000003
:04084000541500004b
:020000040000fa
:1008440070b505000e0018b183690bb900f0dcfa2d
:10085400ab69ac6813b9280000f0d6fa294b9c4266
:1008640019d16c680c23e25e42f200031a4205d1ee
:100874001343a381226e244b13402366a3891b07d1
:1008840001d52369fbb921002800fff767ffd0b128
:100894000120404270bd1d4b9c4201d1ac68e1e790
:1008a4001b4b9c42ded1ec68dce7013b0136a360c4
:1008b400002b04daa269934216db0a2914d02368b8
:1008c4005a1c226019703178a3680029edd1013bcc
:1008d400a360002b0fda22000a21280000f082f81e
:1008e400431cd5d00a20d5e72200280000f07af86e
:1008f400431ce8d1cce70a2023685a1c22601870f4
:10090400c8e7c04674150000ffdfffff9415000020
:040914005415000076
:020000040000fa
:10091800700000201c000000000000000000002003
:100928000c000000000000008c0000200400000003
:1009380001000000100000201000002060000000ee
:10094800010000000000000074150000941500006c
:100958005415000000000000000000000000000026
:10096800000000000000000000000000000000007f
:10097800000000000000000000000000000000006f
:10098800000000000000000000000000000000005f
:10099800000000000000000000000000000000004f
:1009a800000000009000002004000000000000008b
:1009b8009400002004000000000000000c0000204b
:1009c800040000000000000098000020040000005f
:1009d8000000000000000000000000002222222287
:020000040000fa
:1009e800f8b505000e00140018b183690bb900f0c2
:1009f80009fa274b9c4230d16c68a369a360a3898c
:100a08001b0734d5236993b30c23e25e42f200033b
:100a1800f7b2f6b21a4234d023682269981a636989
:100a2800984204db2100280000f01efa28bba368c6
:100a38000130013ba36023685a1c22601f70636960
:100a4800984204d0a389db0719d50a2e17d12100b3
:100a5800280000f009fa90b10fe00e4b9c4201d13a
:100a6800ac68cae70c4b9c42c7d1ec68c5e72100cb
:100a78002800fff771fe0028c6d001267642300014
:100a8800f8bd1343a381226e044b13402366c3e7ca
:100a9800741500009415000054150000ffdfffffd7
:020000040000fa
:100aa800032370b5cd1c9d43083506000c2d1cd2c0
:100ab8000c25a9421bd8300000f045fe254a1468d1
:100ac8002100c1b9244c23681bb9300000f06efd29
:100ad80020602900300000f069fd431c2dd10c2353
:100ae8003000336000f030fe03e0002de1da0c2323
:100af8003360002070bd0b685b1b1bd40b2b03d924
:100b08000b60cc18256003e08c420fd1636813603a
:100b1800300000f019fe200007220b30231d9043ff
:100b2800c31a002be6d05a42e250e3e74b686360f1
:100b38000c00ede70c004968c3e70323c41c9c4381
:100b4800a042dfd0211a300000f030fd431cd9d17b
:0c0b5800c5e7c04690000020940000207b
:020000040000fa
:100b64000222234b1a760022224b1a74224a234b68
:100b74005a62190008224b681a42fcd14121802391
:100b84001e4ad15010008021402243581a42fcd002
:100b9400174b20225a633f221a6318003c21042277
:100ba400435c1342fcd102212c23114ad15410007e
:100bb4003c210222435c1342fcd10d484021032214
:100bc400435c1340032bfbd10d4a0c4b1a621900f2
:100bd40004224b681a42fcd14021b423074ad15065
:100be4001000b421402243581a42fcd07047c0463a
:100bf400001000400014004005010400001c0040e7
:040c040007010200e2
:020000040000fa
:100c080070b5050079b10c1f2368002b00dae418d1
:100c1800280000f098fd1c4a13682bb96360146023
:100c2800280000f091fd70bda34209d92168601821
:100c38008342f3d118685b6841182160eee713001e
:100c48005a680ab1a242fad919685818a0420bd1b9
:100c580020680918581819608242e1d11068526852
:100c6800411819605a60dbe7a04202d90c232b60b7
:100c7800d6e721686018824203d11068526841188b
:0c0c8800216062605c60cbe790000020ff
:020000040000fa
:100c94001e4a1f4b70b50021934203d219700133d1
:100ca4009342fbd1002503261a4803684168b3b96f
:100cb40059b383680c30bbb100230022845c9c547c
:100cc40001328a42fad333000b405a1e93418908f9
:100cd40059188900401803684168002be8d08268dd
:100ce4000c303ab90029e0d059181d7001338b42f9
:100cf400fbd1dae70029e0d133000b405a1e9341bf
:100d04008908591889004018e5e770bd10000020d3
:080d1400000000201809000096
:020000040000fa
:100d1c00f8b51c4b07001e68b36913b9300000f01e
:100d2c006ff84836b4687368013b03d5336833b148
:100d3c003668f7e70c22a55e6db16434f4e7042144
:100d4c00380000f019fb30600028f1d10c230400ae
:100d5c003b602000f8bd01235b42e38120000123ae
:100d6c002566a3812560a560656025616561a56127
:100d7c0008222900583000f0a7fc6563a563a56420
:080d8c00e564e6e740170000f2
:020000040000fa
:100d9400f7b502268b8905000c00334206d02300e8
:100da40047332360236101236361f7bd01ab6a46c6
:100db40000f0aef8009907002800fff773fe30b981
:100dc4000c22a35e9a05f0d41e43a681e7e70d4bdf
:100dd400ab628023a28920601343a381009b20611e
:100de4006361019b4bb10e23e15e280000f000fc1f
:100df40018b10123a2891343a381a0893843a08198
:080e0400d3e7c046c51600004b
:020000040000fa
:100e0c00836913b5040043bb8364c3640365134b4c
:100e1c00134a1b6882620193984201d101238361ba
:100e2c002000fff775ff60602000fff771ffa060e6
:100e3c002000fff76dff0022e0600421606800f0e5
:100e4c00aff801220921a06800f0aaf802221221b1
:100e5c00e06800f0a5f80123a36113bd4017000062
:040e6c00c5160000a7
:020000040000fa
:100e70000b6970b505000c000bb9002070bd18b1ee
:100e800083690bb9fff7c2ff0b4b9c4209d16c6819
:100e90000c22a35e002bf0d021002800fff7d8fb26
:100ea000ece7064b9c4201d1ac68f1e7044b9c4255
:100eb000eed1ec68ece7c046741500009415000014
:040ec00054150000c5
:020000040000fa
:100ec40010b50c4b03b198470b4b03b19847fff790
:100ed400dffe0a4a7f210a4b8b439360094b9847f4
:100ee400094b03b19847094b03b1984700f020f927
:100ef400fee7c046000000000000000000ed00e036
:100f040000000000650f0000000000000000000069
:020000040000fa
:100f140070b50e001d000e23c95e90b014000029a8
:100f240007da00232b60b3891b0611d440f2004377
:100f34000fe001aa00f0c4fa0028f2db4ff200022d
:100f4400029b1340054a9b185a4253412b60ede71c
:100f540040230020236010b070bdc04600e0ffffb6
:020000040000fa
:100f640070b500260c4d0d4c641ba410a64209d18b
:100f74000026fff737f90a4d0a4c641ba410a64259
:100f840005d170bdb300eb5898470136eee7b300c6
:100f9400eb5898470136f2e7f4010000f401000031
:080fa400f4010000f801000057
:020000040000fa
:100fac00002310b5040003604360836081810366f5
:100fbc00c28103614361836119000822583000f03b
:100fcc0083fb054b24626362044ba362044be36214
:100fdc00044b236310bdc0463114000021120000e5
:080fec00b1130000e51600003e
:020000040000fa
:100ff400f7b5050c019393b21f006b439c46140c88
:1010040086b277436643654366443c0ca419a34205
:1010140002d980235b02ed18260cbfb2019b240485
:10102400e41943432000514375195918491903b071
:02103400f0bd0d
:020000040000fa
:02103600fee7d3
:020000040000fa
:1010380010b5054c237833b9044b13b1044800e0cc
:1010480000bf0123237010bd7000002000000000c5
:1010580000000000034b10b51bb10349034800e032
:1010680000bf10bd00000000740000200000000058
:10107800002b11d1002a0fd1002900d1002802d05d
:101088000021c943081c07b4024802a14018029075
:1010980003bdc046a106000003b4684601b5029826
:1010a800fff7b2f8019b9e4602b00cbc7047c046e1
:020000040000fa
:1010b800f7b5040007000026019148340cb9300048
:1010c800febd6368a5680093009b013b009301d5b2
:1010d8002468f3e7ab89012b08d90e22ab5e0133f4
:1010e80004d029003800019b984706436435ebe794
:020000040000fa
:1010f80070b505000c00a8b100f0e0f800200a4a1d
:1011080004210726a04208d0137e0b42fcd0138d81
:101118002b540130538b3342f4d0001b43425841c7
:0c112800c0b270bd0020fce7000c0042cb
:020000040000fa
:1011340010b582b048f200031c68002000f0f0f8fb
:10114400631c0ed084f3888848f204031b6801935f
:10115400019c64086400200021002200230000f0a8
:0c11640095f800f003f8012002b010bd67
:020000040000fa
:1011700010b584b000f082fae1235b0200930023f3
:10118000029302220192039306496846fff7d6f9bb
:10119000054c200000f07cfa40f2e83000f0daf86c
:0c11a000f7e7c0460048e80164160000b4
:020000040000fa
:1011ac001c2101231b04984201d3000c10391b0a8b
:1011bc00984201d3000a08391b09984201d300094f
:1011cc00043902a2105c40187047c04604030202a6
:0c11dc0001010101000000000000000003
:020000040000fa
:1011e8000a4b0b4a1a600b4a9a81c02292025a6033
:1011f8001a00d369002bfcd1044a136802210b435f
:101208001360d369002bfcd17047c046000c004224
:081218000401104141f1ffff48
:020000040000fa
:10122000f8b51f008b8905000c001600db0505d5fd
:101230000e23c95e0022022300f056f9a389054a55
:1012400028001340a38132000e23e15e3b0000f032
:0812500027f9f8bdffefffffd5
:020000040000fa
:1012580070b50c00002519b112b11500022801d98a
:10126800280070bd074b23b11100200000e000bf2b
:10127800f6e716002078013e00f0e3f90134002e6d
:08128800f8d1ede700000000c1
:020000040000fa
:10129000e0b545464e465746e0b45d4620b4254687
:1012a00026462746a046a146a246a346a44684f366
:1012b0000088a44720bcab46e0bcba46b146a8466d
:0212c000e0bd8f
:020000040000fa
:0212c200fee745
:020000040000fa
:1012c4000a4b588b0723184000b97047074b8022fc
:1012d4001a7607225a831b7e5b07f6d5034b04213b
:1012e4001a8d1a7e0a42fbd1efe7c046000c004279
:020000040000fa
:1012f40030b570b179b105004118084a0124137e54
:101304002342fcd02b7813850135a942f7d1012063
:1013140030bd0020fce70120fae7c046000c004283
:020000040000fa
:1013240010b50422094b5a6000f094f800f06af8f2
:10133400fff716fc00f0b4f9fff754fffff7fbf8d2
:1013440000f09af800f0d8f910bdc04600500041f2
:020000040000fa
:10135400094b1b68db439b0700d07047074b996818
:1013640040f2e8335843b0fbf3f0044a93685b1a45
:101374009842fbd8f1e7c04610e000e000000020ee
:020000040000fa
:1013840070b564254a1e55430e0029007031fff7dd
:1013940089fb040040b100212a00016046600c3042
:0c13a400a060643200f094f9200070bddd
:020000040000fa
:1013b00070b50c000e25495f00f096f8a389421c19
:1013c00003d1054a1340a38170bd41f200021343cb
:0c13d000a3816065f8e7c046ffefffff57
:020000040000fa
:1013dc00074a13684bb107491818884202d81060a5
:1013ec001800704701204042fbe7034b1360f2e703
:0c13fc0098000020a0020020a0000020ab
:020000040000fa
:10140800084b04221a6002214222995401224821e1
:101418005a5449215a543321342299540022da6605
:081428007047c046003200408d
:020000040000fa
:1014300070b50c000e25495f00f068f8002803db4a
:10144000636d1b18636570bda389024a1340a381b5
:08145000f9e7c046ffefffffc2
:020000040000fa
:10145800074b00221a819a7901210a439a710222c4
:101468009a70190001228b791342fcd07047c0464c
:04147800000400402c
:020000040000fa
:10147c00064a00231360936047f6ff415160062132
:10148c001160034a936013607047c04610e000e09f
:04149c00000000202c
:020000040000fa
:1014a00070b50500080011000022054c22601a00ea
:1014b00000f03cf9431c02d1236803b12b6070bdde
:0414c0000c000020fc
:020000040000fa
:1014c400002370b5064c050008001100236000f0ed
:1014d4001bf9431c02d1236803b12b6070bdc046c5
:0414e4000c000020d8
:020000040000fa
:1014e80070b50500080011000022054c22601a00a2
:1014f80000f010f9431c02d1236803b12b6070bdc2
:041508000c000020b3
:020000040000fa
:10150c0070b50500080011000022054c22601a007d
:10151c0000f002f9431c02d1236803b12b6070bdab
:04152c000c0000208f
:020000040000fa
:1015300070b5002661b15ab1160048b90c0015000b
:10154000012000f075f8013d20700134002df7d125
:04155000300070bd3a
:020000040000fa
:101554000000000000000000000000000000000087
:101564000000000000000000000000000000000077
:020000040000fa
:101574000000000000000000000000000000000067
:101584000000000000000000000000000000000057
:020000040000fa
:101594000000000000000000000000000000000047
:1015a4000000000000000000000000000000000037
:020000040000fa
:1015b400002370b5054c050008002360fff70cfffd
:1015c400431c02d1236803b12b6070bd0c000020c2
:020000040000fa
:1015d400002370b5054c05000800236000f090f866
:1015e400431c02d1236803b12b6070bd0c000020a2
:020000040000fa
:1015f400002370b5054c05000800236000f088f84e
:10160400431c02d1236803b12b6070bd0c00002081
:020000040000fa
:1016140010b5054b9a6801329a601b6813b1024aef
:0c1624005068984710bdc0460000002030
:020000040000fa
:1016300000b583b000230193012101a8fff75cfdf1
:0a1640000028f9d0019803b000bda6
:020000040000fa
:10164a0000b583b06b46d87101216b46d81dfff7f0
:0a165a004cfe0028f8d003b000bddc
:020000040000fa
:1016640054657374206b6f6d756e696b616365206f
:081674003a2d290d0000c046cb
:020000040000fa
:10167c00034b00229a601a6801210a431a607047d2
:04168c0010e000e08a
:020000040000fa
:1016900010b5034b01001868fff7d4f810bdc04621
:0416a0008c0000209a
:020000040000fa
:1016a400024b02225a6001221a7270470050004114
:020000040000fa
:1016b400401801000200030084468ef3008874473a
:020000040000fa
:1016c40010b50249fff7f6fc10bdc046710e0000cc
:020000040000fa
:1016d40003008218934200d1704719700133f9e76f
:020000040000fa
:0c16e40010b50e23c95efff773ff10bda8
:020000040000fa
:0c16f00042f2000300204b607047c0462f
:020000040000fa
:0816fc00bff35f8f62b6704777
:020000040000fa
:0817040010b500f015f810bd4e
:020000040000fa
:08170c0010b5fff7efff10bd5f
:020000040000fa
:0817140010b500f015f810bd3e
:020000040000fa
:08171c0010b500f013f810bd38
:020000040000fa
:0817240010b5fff703ff10bd33
:020000040000fa
:08172c0010b5fff793fd10bd9d
:020000040000fa
:08173400012040427047c0464d
:020000040000fa
:04173c007047c046ec
:020000040000fa
:041740001000002075
:020000040000fa
:0417440001207047c9
:020000040000fa
:0417480000207047c6
:020000040000fa
:02174c00fee7b6
:020000040000fa
:02174e007047e2
:020000040000fa
:021750007047e0
:020000040000fa
:087e00007fe97fe9f9f756bca8
:020000040000fa
:0200000400807a
:044000007f43ffb14a
:020000040000fa
:0200000400807a
:04400400bbfcffff03
:020000040000fa
:0200000400807a
:0440080080d0f8c0ac
:020000040000fa
:0200000400807a
:04400c00ffffffffb4
:020000040000fa
:0200000400807a
:0440100000000000ac
:020000040000fa
:0200000400807a
:0440140002000000a6
:020000040000fa
:0200000400807a
:0440180000000000a4
:020000040000fa
:0200000400807a
:04401c001e65338466
:020000040000fa
:0200000400807a
:04c00000ff00c0a0dd
:020000040000fa
:0200000400807a
:04c0040000ffffff3b
:020000040000fa
:0200000400807a
:04c008004081e7ddaf
:020000040000fa
:0200000400807a
:04c01000ffffffff30
:020000040000fa
:0200000400807a
:04c01400ffffffff2c
:020000040000fa
:0200000400807a
:04c01800ffffffff28
:020000040000fa
:0200000400807a
:04c01c00ffffffff24
:020000040000fa
:0200000400807a
:04c02000ffffffff20
:020000040000fa
:0200000400807a
:04c02400ffffffff1c
:020000040000fa
:0200000400807a
:04c02800ffffffff18
:020000040000fa
:0200000400807a
:04c02c00ffffffff14
:020000040000fa
:0200000400807a
:04c03000ffffffff10
:020000040000fa
:0200000400807a
:04c03400ffffffff0c
:020000040000fa
:0200000400807a
:04c03800ffffffff08
:020000040000fa
:0200000400807a
:04c03c00ffffffff04
:020000040000fa
:0200000400807a
:04c04000ffffffff00
:020000040000fa
:0200000400807a
:04c04400fffffffffc
:020000040000fa
:0200000400807a
:04c04800fffffffff8
:020000040000fa
:0200000400807a
:04c04c00fffffffff4
:020000040000fa
:0200000400807a
:04c05000fffffffff0
:020000040000fa
:0200000400807a
:04c05400ffffffffec
:020000040000fa
:0200000400807a
:04c05800ffffffffe8
:020000040000fa
:0200000400807a
:04c05c00ffffffffe4
:020000040000fa
:0200000400807a
:04c06000ffffffffe0
:020000040000fa
:0200000400807a
:04c06400ffffffffdc
:020000040000fa
:0200000400807a
:04c06800ffffffffd8
:020000040000fa
:0200000400807a
:04c06c00ffffffffd4
:020000040000fa
:0200000400807a
:04c0e000ffffffff60
:020000040000fa
:0200000400807a
:04c0e400ffffffff5c
:020000040000fa
:0200000400807a
:04c0e800ffffffff58
:020000040000fa
:0200000400807a
:04c0ec00ffffffff54
:020000040000fa
:0200000400807a
:04c0f000ffffffff50
:020000040000fa
:0200000400807a
:04c0f400ffffffff4c
:020000040000fa
:0200000400807a
:04c0f800ffffffff48
:020000040000fa
:0200000400807a
:04c0fc00ffffffff44
:00000001FF
